:020000000F28C7
:10000800FE00030EF1000408F2000A08F300831250
:100018007F08F400E22835298B01703083169F0091
:1000280001309100013083129F00F930831692004D
:1000380005308312920093010C309500013083162D
:100048008500831285018316870183128701843016
:10005800831681008312A001A201A1017D30A400B2
:100068002408A800A301063081008B168B173C28B2
:10007800A208031D4028412846280230A40024086D
:10008800A20046280130102183129F144B289F1884
:100098004E284F284B2850281E08A4002408A000EA
:1000A800A008031D582859285F2820080138A400F3
:1000B8002408A0005F28200893002208013A031DA5
:1000C800662867283C28A201A108031D6C286D2812
:1000D800A628F130A4002408A700A601A60A093022
:1000E8002602031C782879287B289D289D288711BB
:1000F800271C7F288028822807168428071284282E
:100108002708A4000310240CA5002508A700203008
:100118002A218312871520302A2183128711013062
:10012800A4002408A60709302602031C9C289D2841
:100138007B28071520302A21831207118710A10177
:10014800A10A3C289E30A4002408A700A601A60AFC
:1001580009302602031CB128B228B428D628D6288C
:100168008711271CB828B928BB280716BD280712ED
:10017800BD282708A4000310240CA5002508A70003
:1001880020302A218312871520302A2183128711D3
:100198000130A4002408A60709302602031CD5282C
:1001A800D628B428071520302A2183120711871072
:1001B800A1013C283C283C283C280F280B1DE52899
:1001C800E62805290B11063081000130A802A8088D
:1001D800031DEF28F028FA287D30F0007008A800E9
:1001E8000430F0007008A300A201A20A2308031D2E
:1001F800FE2802290130A302071405290710052942
:1002080005297408FF0073088A0072088400710EBB
:100218008300FE0E7E0E0900F70022290430F60046
:100228007608F8001A2952302A211A290130F802D2
:10023800031D1F2920291729222922290130F70205
:10024800031D27292829122929290800F5002D2905
:100258002D290130F502031D322933292D2934298E
:0E0268000800A001A101A201A301830110283A
:02400E00E1F3DC
:00000001FF
